:10014000021D800A0A5052494E540D0A80140A506A
:1001500052494E540D0A801E205052494E542022BE
:10016000544154544C4554414C45204D4F44454C0A
:100170002023223B0D208028105052494E54204D00
:100180004F44454C0D1080320A5052494E540D0ACE
:10019000803C225052494E5420222020532F4E2082
:1001A000222C20534E25313030303030303030303A
:1001B0000D2280462A5052494E542022284329209D
:1001C00031393839204F4E53455420434F4D505507
:1001D00054455220434F52502E220D2A80500A502F
:1001E00052494E540D0A805A2F5052494E542022E3
:1001F0005454424153494320222C564552532F31E7
:1002000030302C222E222C2330322C5645525325AE
:0D0210003130300D2F8064084E45570D0829
:10C000008E00FFBDF6A78621BDFB6EBDC0C842C035
:10C010002743C03044C03946C07B4DC12B50C29F1E
:10C0200052C27653C0AA00BDFB6E717F147EFBC561
:10C03000BDFB6EBDF6A77EC706BDC0E33CBDFD06D9
:10C04000BDFB93383CC610A600BDFD0BBDFB970899
:10C050005A26F4BDFB9338C610A60081202C028618
:10C060002E817F2F02862EBDFB6E085A26EBBDF671
:10C07000A7BDC128812E26C47EC000BDFB6EBDFBBE
:10C0800097BDC0F6183C862CBDFB6EBDC0F6DD56D4
:10C09000862CBDFB6EBDC0F637BDF6A73238A700B3
:10C0A000089C5626F9A7007EC000BDC0E3BDFD0672
:10C0B000BDFB93A6009753BDFD0BBDFB93BDC0F622
:10C0C000E700BDF6A70820E5383CBDC128A1002740
:10C0D000096D0027F308080820F3333336EC011804
:10C0E000326E00BDFB6EBDFB977F00527F0053BDDB
:10C0F000C0F6187EF6A7BDC128812E26037EC0009B
:10C10000810D2603DC5239803025EB810A25088019
:10C110000725E3811024DF9746BDFD13DC5205059A
:10C120000505DB46DD5220CE7EFB31BDFB6EBDF644
:10C13000A7BDFAFC26FB71F8175FF740005CC10849
:10C1400027057C001720F371F8175FF140002738AE
:10C15000B64000363771F817CEC1754FBDF528329D
:10C160008A30BDFB6ECEC17D4FBDF528328A30BD11
:10C17000FB6E7EC0003A2042414E4B2000205245CB
:10C1800041445320415320005CC10827057C00171F
:10C1900020B971F817CE4002EF001805847F8B405C
:10C1A000188C400026F2CE4002AC002743DF46EE5A
:10C1B00000DF4871F817BDF6A7CEC1E14FBDF528E5
:10C1C0009648BDFD0B9649BDFD0BCEC1E64FBDF5B2
:10C1D000289646BDFD0B9647BDFD0B71F8177EC036
:10C1E0000053454520002041542041444452200042
:10C1F0001805847F8B40188C400026AD8601974639
:10C2000071F81796179A469717CE40004F5FED00CA
:10C21000EC00261E4353ED00A300261F08088CC027
:10C220000026EB7C00469646810826D771F8177EDB
:10C23000C000CC0000ED00EC002007CCFFFFED00BB
:10C24000EC003C373671F817BDF6A7CEC26B4FBD78
:10C25000F528323318BDFD068640BDFB6E383CBD67
:10C26000FD0638EC004353ED0020F84249542045C8
:10C2700052524F522000BDFB6EBDF6A74F363236EC
:10C28000BDF727DE56BDFD06BDFB93324C3681401F
:10C290002709840726E8BDF6A720E3327EC000BD4B
:10C2A000FB6EBDF6A77F0053BDC0F6C43F37BDFB94
:0DC2B00093BDC0F6DD5632BDF7717EC000B3
:10C4000000000030303030303030303030300D54BB
:10C410004154544C4554414C45204D4F44454C20CB
:10C420003220202843292031393839204F4E5345B6
:10C430005420434F4D505554455220434F52502E97
:10C440000D4C495354CB34545952554ECAD25052C4
:10C45000452A52554ECACB462452454D494E44CFEB
:10C46000B3465245D767414F4E454F4ED80A4141DA
:10C4700041454F4646D80542424E455854C950544E
:10C480004F4C4554CE975641524946CDDB4E4F5402
:10C4900045474F544FCB1C454E474F535542CD86D1
:10C4A0005352455455524ECDAF464F52C8C84745DA
:10C4B000544255525354CEA75853544F5245CEED83
:10C4C0004150534554D3AE564150434C52D4185466
:10C4D0004553444FDADE31313143414C4CDC0932B3
:10C4E00032434F554E54DD6745534C454550D3308C
:10C4F000525550524F47DBA15855474554D5054436
:10C5000046544F4E45D78252535553454E44D47CE2
:10C510002F4F4E455252D6632352415445DD40546D
:10C520005941534DDFBC4A4E4B52454DCDCC415243
:10C530004B5052494E54CC6553584D4954D83257FC
:10C540004F53544F50CAC5544F4954455854D6833D
:10C550004F4F54455854D71F475354494D45D84F12
:10C56000405254494D45D9A54041444C4F4F50DEAF
:10C57000CD5653544F5245DC8C56474554DCC63398
:10C5800033494E505554CE0038585348414B45D846
:10C59000154F46464C44D16C454F4E4C4F4144DDFF
:10C5A000A544494DDCF85245414E4557CAB14F4C60
:10C5B00044434F4EDD1A444545CE91544FC8EB4697
:10C5C000524F4DF38A53544550C9004154C9064354
:10C5D00048414EE67E5459474554E6AC26474F50F5
:10C5E000494EE72A544845534449EA8020202050C8
:10C5F0004552494F44EB67414253E6694245455332
:10C600005152E7AB47415454454D50E845484953D2
:10C61000494EE9094F46464153494EE9754E554347
:10C620004F554E54EAD3454C4F47EC1F494E4745B2
:10C630005850EDDA49524556455253EA695A595312
:10C640004EEA7550495A454D4F44454CEA6053E611
:10C65000353DE4BB252F2F2A343E3DE48C2F233C6F
:10C660002F3E3CE4977E2F2A3C3C3EE4972B3D2D09
:10C670003E3EE4A9454E442E2E3C3DE4B23F2F3EC3
:10C680003E3CE4C23C3E3C0404E4C98EBFFF7F0054
:10C69000760E86FF9791BDFACF861A97111A1ABDAA
:10C6A000FACF4FCE738C6F00088C73A226F87F00F0
:10C6B000B37F00B4CC0C00FD72887F00B57F006AA8
:10C6C0007F0076860AB7B59ACC1770DDAF863997AA
:10C6D0009F9797979497A597A897A2867E97ABCC9C
:10C6E000FB6EDDACCC0000DD9ADD9C7F0077BDF6F3
:10C6F000A786FF978C979E7F00927F00B67F00935E
:10C700007EC84B4F4B0D8EBFFF86FF979E860AB7A4
:10C71000B59A7F00817F008CBDF6A7CEC7034FBDC1
:10C72000F528CEC729FF738CCE0000FF7394FF73EA
:10C730008E863EBDFB6E4FCEB294BDF438083CCE23
:10C74000B294865CBDEEE0261EBDE407FC72189331
:10C75000522607FC721A935427033820D4865CBDF6
:10C76000EEE027037EF38A1838DF5618BDEF65DC4C
:10C7700056DD4EBDEEF0DC522634DC54261B8627F7
:10C78000BDEEE027AC7EC87A45444954494E472067
:10C7900044495341424C45440D7D0092270DCEC77C
:10C7A000884FBDF528BDF6A77EC7314D2A06CC00BF
:10C7B000087EF0040909098A80ED00DF46DC4E930B
:10C7C00046E702DE4E09E700FE73A209FC73A2E011
:10C7D00000820018EC00847F9354FE73A22505BDEF
:10C7E000F4A52705FF73AE201BFF73A6FF73AEFCF5
:10C7F00073A2FD73A8BDF4C9FF73A4BDF619FC7341
:10C80000A6FD73A2DC4E9346C10526037EC731FE0A
:10C8100073A2FF73AAF373AAFD73AC188CB28F18BE
:10C8200023037EF42FFD73A2BDF632FC73AEFD73BD
:10C83000A6DC4EFD73A8DC46FD73A4BDF6197EC7C9
:10C8400031CE01006F000926F8203AFEB5CD8C30BC
:10C85000392722B6C42E815326E7CE0142FF73A4A6
:10C86000CE73D2FF73A6FC0140FD73A8BDF619FC80
:10C8700073A6FD73A27ECACE0000CCC878FD738C6F
:10C88000CCC441DD520908A600B1C42B27F8DF460D
:10C89000A6003CDE52E6002B2811270B18C3000827
:10C8A00018DF5220F0DE4A08E600DF4A38083CE193
:10C8B0000027F2C180240838DE463CDE5220DDDE4F
:10C8C0004A08A60038363739BDF672BDF342DC524D
:10C8D000FD7394B6C42C814F2709FC739483000424
:10C8E000FD7394CCC5BBDD527EC885BDE407DC5426
:10C8F000FD7398DC52FD7396CCC5C5DD527EC885AC
:10C90000BDE4077EC90FCC0001DD545F4FDD52DC72
:10C9100052FD739ADC54FD739CFC738CFD739EFF77
:10C9200073A030200518C3000E18EC00271C18BC9B
:10C9300073941826F0FF73AA18C3000EFD73AC3071
:10C94000FF73AEBDF632FE73AC35FE73A07EEEF71C
:10C95000BDEEFD24037EF38AFD73903CFE739426A6
:10C9600004387EF38ABC7390270738BDF64B7EC926
:10C970005BEC02F3739CED02EC00F9739BB9739AC4
:10C98000295BED00FC739A2B267D73962A066D00B9
:10C990002A4D20046D002B39EC0018BC739625310C
:10C9A000263D18EC0218BC73982526272420307DDC
:10C9B00073962B066D002B2720046D002A13EC00C4
:10C9C00018BC73962519260918EC0218BC73982513
:10C9D0000E38FC739EFD738CFE73A02006ED0038AC
:10C9E000BDF64B7EEEF7BDE407DC522605DC544D68
:10C9F0002A09CC00087EF0047EF38A3637862CBDE7
:10CA0000EEE026F4BDE407DC5226E7DC544D2BE2D1
:10CA10003332DD48DC54934825D83CFE738CEC005F
:10CA2000847FDD502733189C48252E9C54270224F0
:10CA300028BDF6A7CECA3F4FBDF528387EC70643AE
:10CA4000414E4E4F5420455241534520435552527A
:10CA5000454E54204C494E450DDE54DF52DE48DF32
:10CA600054CE73D2BDF4B72404387EEEF7FF73A61C
:10CA7000DC52C30001DD54BDF4B72408FC73A6FDED
:10CA800073A22012FF73A4FE73A2FF73A8BDF61950
:10CA9000FE73A6FF73A2DE5027CFDF54CE73D2BD44
:10CAA000F4B7080808A600810D27BF813A27BB20EC
:10CAB000F3BDEEF0810D2707813A27037EC9E6CC4E
:10CAC00073D2FD73A2BDF37F7EC706BDF37F86FFE1
:10CAD0002004BDF37F4F978C7F0081CE73D27F00FF
:10CAE000547F0055BDF4B724037EC706FF738C96B0
:10CAF000B5271BBDFB6EEC00847FDD547F00527FA9
:10CB0000005386019745BDF563863EBDFB6E080860
:10CB100008BDF6B8CCC479DD527EC885BDE4073CBB
:10CB2000BDF37FBDF4DC270738CC00157EF004325E
:10CB3000327ECAECBDEEFD24037ECBD13CFD73AA50
:10CB400018EC00DD64EC02DD66CCF0CEDDAC387FA5
:10CB500000547F0055862CBDEEE0260DBDEF65DC50
:10CB6000522706CC00087EF004DC542BF6363796AC
:10CB7000442729862CBDEEE0270A862DB1C42EBDA0
:10CB8000EEE02613BDEF6596442711DC5226D4DC77
:10CB9000542BD0DD5E200ACC00002003CC7FFFDDCB
:10CBA0005E3332DD543CBDF4A52512BDF5F4BDF471
:10CBB000B7250AEC00847F935E27F025EEFE73AA6A
:10CBC000DC64ED00DC66ED02CCFB6EDDAC387EC7CC
:10CBD00006BDEF65DC522706CC00087EF004DC546D
:10CBE0002BF6363796442729862CBDEEE0270A8699
:10CBF0002DB1C42EBDEEE02613BDEF65964427117E
:10CC0000DC5226D4DC542BD0DD5E200ACC00002080
:10CC100003CC7FFFDD5E3332DD5496763686019796
:10CC2000763CBDF4A52517BDF5F47D0093262ABDFD
:10CC3000F4B7250AEC00847F935E27EB25E93832B0
:10CC400084019776863BBDEEE0260BBDFB31811358
:10CC500027F9811127F57EC706383284019776BD02
:10CC6000FACF7EC706863BBDEEE026037EEEF78652
:10CC70000DBDEEE0270C863ABDEEE027058D0A7E5D
:10CC8000EEF709BDF6A77EEEF786019745BDF53CA8
:10CC900027698623BDEEE02639C600A6008130262E
:10CCA00002C680D745BDE4079655847F9A459745CF
:10CCB0008648C610A10027138642C602A100270B92
:10CCC0008651C608A1002703C60A0908F7B59A7E4F
:10CCD000CCFBA600815C260A08BDE40796559DABF7
:10CCE0002019867BBDEEE0260CBDCD20867DBDEEF5
:10CCF000E026252006BDE407BDF563862CBDEEE0E9
:10CD0000278B863BBDEEE0260139860DBDEEE02780
:10CD10000A863ABDEEE027037EF38ABDF6A70939FD
:10CD2000BDE407BDCF8CDC523637DC543637862C59
:10CD3000BDEEE026E3BDE407BDCF8C3332DD4833E2
:10CD400032DD469352250E2706CC00167EF004DC19
:10CD500054934825F4BDCD6FBDF11ABDCD6F9DAB89
:10CD6000DC46935225EF2606DC54934824E7393CF1
:10CD7000DE463CDE483CDE64DF46DE66DF4838DF08
:10CD80006638DF643839BDF672BDE407BDF37F3C19
:10CD9000BDF4DC270738CC00157EF00418FE738C38
:10CDA0003CFE738E3C7F7394BF738E187ECAECBDBD
:10CDB000F37FFC738E26037EF38ABE738E38FF7377
:10CDC0008E38FF738C38BDF64B7EEEF7FE738C7F8A
:10CDD00000547F0055BDF4C97ECAE7BDE407DC52AC
:10CDE0002604DC5427037ECB11BDF4D325037ECA71
:10CDF000EC7EC706BE739238FF738C3838BDF6A739
:10CE00003CBDF53C2609BDEEFDDD54256820233CE4
:10CE1000BDEEFDDD5424037EF38AA600B1C42D9738
:10CE2000454FA70038BDF528964509A700863ABDAD
:10CE3000FB6E3CFE738C3CCEFFFFFF738CBF739286
:10CE4000DC543736863ACEB394BDF438CEB394A6CC
:10CE500000810D2606A7018630A700BDE407BDEEC0
:10CE6000F0810D268F380FDC54ED02DC52ED000E00
:10CE700038FF738C3832B1C43132863BBDEEE027C7
:10CE800003BDF6A7862CBDEEE026037ECE007EEE27
:10CE9000F7A600810D270ABDF342862CBDEEE027E0
:10CEA000F67EEEF77EF38ABDCF73862CBDEEE026CC
:10CEB000F3BDE4073CDE522609DE5427058C000949
:10CEC000250738CC000B7EF004183837C601D7523E
:10CED000862CBDEEE0260DA600803025C7810324F8
:10CEE000C3975208323CD652BDF96A202CBDCF738D
:10CEF00086319762862CBDEEE0261D8623BDEEE0CE
:10CF00002631A600088132270B813427078131277B
:10CF1000037EF38A976220DC3CFE73AAB6C42D819F
:10CF20004E2704DC422002DC66ED02DC64ED0038B2
:10CF30007EEEF7BDEEF08127270481222610CCF08B
:10CF4000CEDDACBDCC89CCFB6EDDAC7ECF18BDE4B4
:10CF500007D662C134260C9652BDF0CE9653BDF072
:10CF6000CE2004C13226059654BDF0CE9655BDF0B4
:10CF7000CE2081BDEEFD2511FD73AA3CFE73AAEC07
:10CF800000DD64EC02DD6638397EF38ACC0003DD17
:10CF900046CC8000D39CDD48DC46D99B999A9352BD
:10CFA000250B2608DC4893542503270139CC0016AD
:10CFB0007EF0043CFC73A28373D22604387EEEF725
:10CFC000188C3EBF2522CECFD04FBDF5287EC70698
:10CFD00050524F4752414D20544F4F204249472015
:10CFE000464F5220524F4D0018C30142FD73D0CE20
:10CFF000D3034FBDF528BDF6A7CE177096431A91FF
:10D000004327FBBDFAF7260D0926F1CED3134FBDFA
:10D01000F5287EC706BDFB31811826037EC7068131
:10D020001526D9CEB601DF5286019755FC73A2DDD5
:10D030004ACC8D70DD4CCE73D0BDD07638862BBDFA
:10D04000EEE03C260C4F5FDD4CDD4ACEC000BDD08B
:10D05000764FCED061A60081242714BDD0F80820D9
:10D06000F43A303030303030303030300D0A24BDBA
:10D07000D149387EEEF7DF4E7F00467C0046089CA3
:10D080004A27069646811026F2863ABDD0F87F00E0
:10D09000479646BDD0D7DC4ED34C37BDD0D732BD36
:10D0A000D0D74FBDD0D7DE4EA600BDD0D7089C4A02
:10D0B00027107A004626F14F9047BDD0D7BDD0CC7F
:10D0C00020B44F9047BDD0D7BDD0CC39860DBDD050
:10D0D000F8860ABDD0F839369B47DD4732364444DE
:10D0E0004444BDD0EA32BDD0EA39840F8B30813A56
:10D0F00025028B07BDD0F8393CDE52A7008CB680E4
:10D10000270608DF5238393CCEB601DF524F97541C
:10D110008601BDFB6E9655BDFB6E43BDFB6EA60042
:10D12000BDFB6E9B549754088CB68126F19654BD76
:10D13000FB6EBDFB31811527CF810627078118269D
:10D14000C77EC7067C00553839DE528CB681270B66
:10D150006F00088CB68126F8BDD1078604BDFB6E32
:10D16000BDFB31811827DA810626DE39BDE407BD13
:10D17000CF8CDC52DD64DC54DD66862CBDEEE0270E
:10D18000037EF38ABDE407BDCF8CBDD2F82406CC64
:10D1900000167EF004B6C42E81532708DC529A4054
:10D1A000DA41DD5218DE523CDE543C18862CBDEECE
:10D1B000E02707CC177036372020BDE407DC522764
:10D1C00006CC00177EF004DC543637862CBDEEE02A
:10D1D0002608BDEEFD24067EF38ACC004EDD4E33DC
:10D1E00032DD501838DF5438DF52183CDE4E8C00E8
:10D1F0004E260ACED3034FBDF528BDF6A7BDD216E5
:10D200002626DE4E8C004E260ACED3134FBDF528BF
:10D21000BDF6A77ED2EADE5096431A914327FBBDA6
:10D22000FAF726030926F139BDFB31811826037E62
:10D23000D2EA811526C78601974720347C0047BD76
:10D24000D216260D3338BDD2F824037ED2CA7ED240
:10D25000EABDFB31333881062716811826037ED2BA
:10D26000EA811527043C3720D6DF66D7657A004768
:10D27000BDD2F8254BDE663CD665377F005A7F006D
:10D280005B8601BDFB6E9647BDFB6E43BDFB6EBD6D
:10D29000D2F82515965A8180271EBDF11ABDFB6E66
:10D2A0009B5B975B7C005A20E6965A818027094F4A
:10D2B000BDFB6E7C005A20F1965BBDFB6E7ED23CBE
:10D2C0008604BDFB6EBDD21626197300647300651B
:10D2D000DC664353C30001DD66DC64C9008900DD00
:10D2E000642007BDFB31810626D6DE4EDC64ED00EE
:10D2F000DC66ED02387EEEF7965390652604DC542A
:10D3000093663957414954494E4720464F52204E63
:10D31000414B004E414B204E4F5420464F554E44FA
:10D32000204245464F52452054494D454F555400E3
:10D33000BDE407DC522706CC00187EF004DC54263E
:10D340000D96431A914327FB4FDD6C7EEEF7DD6EA1
:10D35000200108A600B1C43127F8813A272C810D9D
:10D3600027283C20091ADC6C936E270B24097B408C
:10D370001527F2387ECB11DD6C38CC0000DD54BDB2
:10D38000F4D325037ECAEC7EC7063C1ADC6E936C90
:10D39000270925022AF5862ABDFB6ECE0000DF6C28
:10D3A000387EEEF79DA53838CC000C7EF004BDE445
:10D3B00007DC52270DCC000C7EF0043C8DE6387E55
:10D3C000EEF7DC544D26F4C10E24F0C10824178674
:10D3D000805D2704445A20F9369A159715329A8BA6
:10D3E0009720978B201EC00886805D2704445A2012
:10D3F000F9B1C43124024444369A039703329A8A1D
:10D400009701978A862CBDEEE027A37EEEF79DA8B4
:10D410003838CC000C7EF004BDE407DC52270DCC7C
:10D42000000C7EF0043C8DE6387EEEF7DC544D2691
:10D43000F4C10E24F0C108241886805D2704445AE4
:10D4400020F9364394159715329A8B9720978B20A5
:10D4500021C00886805D2704445A20F9B1C43124D4
:10D46000024444364394039703329A8A9701978A79
:10D47000C00E862CBDEEE0279F7EEEF7BDD5F5866B
:10D48000809A8A9701978ABDEEF08122270481272E
:10D490002610CCD4D8DDACBDCC89CCFB6EDDAC7E07
:10D4A000EEF7BDD63DDC7B2604DC79271BBDF11AE7
:10D4B000BDD4D8DC7B830001DD7BDC79C200820037
:10D4C000DD7926E9DC7B26E53CFE73AADC64ED0011
:10D4D000DC66ED02387EEEF73CDE7D8C0113240124
:10D4E0000FBDD5EF717F03BDD5EFC608442505718B
:10D4F0007F0320057280032000BDD5EF5A26ED7210
:10D500008003380E39BDD5F5BDD63D862CBDEEE085
:10D5100027037EF38ABDE407DC7B2607DC7926033C
:10D520007ED4C886FE948B9720978B867EB7010C9D
:10D53000CCD596FD010DDC522706CC00257EF004EB
:10D540000FDC42D354DD54DC40D9539952DD52965E
:10D55000AE8900974E7F007FDF467F0080DC7D83B1
:10D56000011325037A00800E01010F7201140E1AB7
:10D570000F967F2616964E90AE251026EADC529323
:10D5800040250826E2DC54934224DC71FE140E860A
:10D59000FF97807ED4C871FE14968027010ED6179F
:10D5A00037C4F7D717DC7D04D37D18BDD5F1C6800D
:10D5B00096150425070101BDD5EF20F417DE46BD01
:10D5C000F0CEDC7B830001DD7BDC79C2008200DDF4
:10D5D00079DC7D04047B0115260583000126F6DC39
:10D5E000792608DC7B260486FF977F33D7173BDE3E
:10D5F0007D0926FD39BDE4073CDC52DD46DC54DD07
:10D6000048BDF083CC04B07B01BB2703CC0960DDAF
:10D6100053BDF14ADC52260CDE548C0FA024058C3D
:10D62000001E240A38CC00197EF0047EF38A188389
:10D630000007DD7D38862CBDEEE026EF39BDE4071E
:10D64000DC52DD79DC54DD7B862CBDEEE026DCBDD2
:10D65000EEFD25D7FD73AA3C18EC00DD64EC02DD7D
:10D66000663839BDE407BDF37F3CBDF4DC270A38DA
:10D670007F0081CC00157EF004DF823886FF978121
:10D680007EEEF7BDCF73860DB773AC862CBDEEE092
:10D690002616865CBDEEE02636BDE4079655B773C8
:10D6A000AC862CBDEEE027273C4FCEB394F673AC8E
:10D6B000BDF43ACEB394A600B173AC270C08DF5288
:10D6C00038BDF0CE3CDE5220EDBDF0CE7ECF19BD90
:10D6D000E407DC522706CC001A7EF004DC54273223
:10D6E000DC54DD52BDFAF7270FBDFB3136BDF0CE5D
:10D6F00032B173AC271920E896431A36BDFAF732D7
:10D7000026E7914327F4DC52830001DD5226E97EAF
:10D71000CF18BDFAF727F8BDFB31BDF0CE20F0BD24
:10D72000CF73860DB773AC862CBDEEE02612865CF7
:10D73000BDEEE027037EF38ABDE4079655B773ACD0
:10D740003CBDF11AB173AC2705BDF6A920F33836FC
:10D75000863BBDEEE032270C810D2605BDF6A720E5
:10D7600003BDFB6E7ECF18BDF37FCCB28FB373A227
:10D77000DD547F00527F005386069745BDF5637EDA
:10D78000C706BDE407DC522706CC001B7EF004DC94
:10D7900054188C00DC1825F13637862CBDEEE026B7
:10D7A000E8BDE407DC5226E1DC54260432322035A1
:10D7B00005DD5425D43332DD463C867EB70106CCE8
:10D7C000D7E8FD010771FD039608DC09D346DD0BA0
:10D7D0008601970F860897081ADC4626FB7F00080B
:10D7E0008600970F387EEEF79608DE54270E09DF85
:10D7F0005488019708DC0BD346DD0B3BDC0BD3468A
:10D80000DD0BDF463B86FF3620024F36BDF37F320D
:10D8100097927EC706BDE407DC522706CC001C7E2B
:10D82000F004DC542706DDAF860120014F97767E99
:10D83000EEF7A600812D260DBDFAFC26FB86FF081B
:10D8400097777EEEF7812B27037EF38A4F20F0B681
:10D8500073B0BA73B1BA73B4BA73B5BA73B8BA73F2
:10D86000B9BA73BCBA73BDBA73BEF673BF271FC112
:10D870002025028AFFBA73C0BA73C1BA73C2F673A5
:10D88000C3270BBA73C4BA73C5BA73BE2706CC00DC
:10D89000267EF0047F004A7F004BFC73B2DD4CCC47
:10D8A000003CDD484F5FDD46DD52FC73B6DD54BD04
:10D8B000F27EBDD98A4F5FDD46DD52CC0E10DD54BD
:10D8C000FC73BADD48BDF27EBDD98A4F5FDD465C90
:10D8D000DD52F673BF5ADD48CC5180DD54F673C774
:10D8E000C1292404CB142008C0502515C1142411CB
:10D8F000D75E54545C4FD348DD48F673C3C10D2541
:10D9000006CC001D7EF004D7463CCED999C1032435
:10D9100009D65EC40326037A00495F7A00462707CA
:10D92000EB0089000820F438D348DD48BDF27EBD05
:10D93000D98A4F5FDD52D65EDD54CC01E1DD46CCA5
:10D940003380DD48BDF27EBDD98ABDEEFD250E3C9B
:10D9500018DC4AED00DC4CED02387EEEF7DC4CDDE5
:10D96000484FD64BDD465FDD52C664DD54BDF27EC6
:10D970000FDC50DD42D64FD7418664D64A3DDB4EA0
:10D980008900D74097AE0E7EEEF7DC50D34CDD4CCD
:10D99000DC4ED94B994ADD4A391F1C1F1E1F1E1F22
:10D9A0001F1E1F1E1FBDEEFD3C24460F96AE975254
:10D9B000DC40DD53DC4297550ED75ECC0064DD4879
:10D9C0005FDD46BDF14ADC53DD5F965597619651A8
:10D9D000D65EDD544F5FDD52DD46C664DD48BDF1E5
:10D9E0004ADC549B61DD54DC5FC9008900DD5220B4
:10D9F0000918EC02DD54EC00DD52188C800025077C
:10DA000038CC001E7EF004CC0001DD46CC5180DD18
:10DA100048BDF14ADE543CDC4EDD52DC50DD544F53
:10DA20005FDD46CC0E10DD48BDF14ADC54FD73BA13
:10DA30005FFD73B8DC4EDD52DC50DD544F5FDD46D8
:10DA4000CC003CDD48BDF14ADC54FD73B65FFD738C
:10DA5000B4DC50FD73B25FFD73B038187F00527AAA
:10DA600000527C0052BDDACE260A83016E24F3C335
:10DA7000016E200883016D24E9C3016D3637D6524B
:10DA8000CB50C1642502C0644FFD73C65FFD73C4F3
:10DA90003332CED9997F00547F00537C005337E650
:10DAA00000BDDACE260937D653C1023326015C0801
:10DAB000D75533935424E4D3544F5CFD73BED653EF
:10DAC000FD73C25FFD73BCFD73C0387EEEF7369602
:10DAD0005284033239CC00207EF0047EF38ABDEEFE
:10DAE000F08122270481272613BDDB8DCCDB70DD7E
:10DAF000ACBDCC89CCFB6EDDAC7EEEF7BDE4071887
:10DB0000DE523CDE543C18862CBDEEE026CDBDE452
:10DB100007DC5226C0965426BCD6552750C1212476
:10DB2000B4BDDB8DD7461838DF5438DF5218D646DF
:10DB300086209046270F7800557900547900537954
:10DB400000524A20EF7B80522705720403200371A4
:10DB5000FB0372041571FB157800557900547900A8
:10DB6000537900525A26DE72201571DF157EEEF7CA
:10DB7000C608492405720403200371FB03720415CF
:10DB800071FB155A26EC72201571DF153986049A3F
:10DB90008A9701978A86249A8B9720978B71DB1539
:10DBA000398627BDEEE0270A8622BDEEE027037EF8
:10DBB000F38ABDDBDD974EBDDBDD36BDDBDD163226
:10DBC000DD46BDDBDDBDDBDDD64E270E5AD74E3C34
:10DBD000DE46A70008DF463820EB7EEEF78D0A48C8
:10DBE000484848368D03331B39A600088030250C81
:10DBF000810A250B80072504811025037EF38A39CD
:10DC0000CC00217EF0047EF38ABDE407DC5226F0CE
:10DC1000DC54183C18862CBDEEE026EABDEEF081FF
:10DC200022270481272610183818DDACBDCC89CCFA
:10DC3000FB6EDDAC7EEEF7BDE40718DE523CDE5431
:10DC40003C18862CBDEEE02705CC004E2005BDEE2D
:10DC5000FD25B3FD73AA1838DF5438DF5238DF468C
:10DC6000183CBDFAFC26FBCEDC733CDE463CDC54A3
:10DC7000DE52393CFE73AAED02183818ED00387EEA
:10DC8000EEF77EF38A38CC00247EF004BDEEFD254D
:10DC9000F13C188C719C25EDEC00DD56EC02DD5456
:10DCA000188372184353C30001541736BDF771DC53
:10DCB00054DD56324CBDF771387EEEF77EF38A386C
:10DCC000CC00247EF004BDEEFD25F13C188C719C47
:10DCD00025ED3C188372184050C30001541736BD1F
:10DCE000F727DC56DD52324CBDF72738DC56ED0203
:10DCF000DC52ED00387EEEF7BDE653DC522615DC33
:10DD000054188C0014250C8C0C01240718FD728803
:10DD10007EEEF718CC00237EF0047F00B37F00B4C2
:10DD2000867BBDEEE0260EBDEEFD250CDDB3867DC7
:10DD3000BDEEE026037EEEF77EF38AC6317EF00468
:10DD4000BDE407DC5226F4DC5427F04D26EDD7B7AE
:10DD500086C05F5C90B724FB5A7B01BB2601545AF6
:10DD6000D71CD7637EEEF77F0008BDEEFD251CFDB6
:10DD7000B598867EB70109CCDD8EFD010AC602D7B3
:10DD800008D608DC0DDC09C612D7087EEEF7960827
:10DD9000FEB598EC02C30001ED02EC00C900890059
:10DDA000ED00DE0D3B86FF974F860197503CCC007F
:10DDB00052FD73ACBDEEFD25123637862CBDEEE06C
:10DDC00026073332FD73AC2002323338BDE407DC62
:10DDD00052DD64DC54DD66862CBDEEE027037EF365
:10DDE0008ABDEEFD25F8FD73AA3C96B636861897D7
:10DDF000B6BDFACFCE006496431A914327F9BDFA17
:10DE0000F726EE0926F18615BDFB6E7C004FD64F36
:10DE1000C11426208618BDFB6EFE73AA4FED025F6B
:10DE2000ED00FE73ACDC66ED02DC64ED003297B60B
:10DE3000387EEEF7BDDEB927CDBDFB318118260453
:10DE4000C61520D5810426098606BDFB6ED64F2057
:10DE5000C88101269CBDDE6426978606BDFB6E7CCC
:10DE6000005020D0CEB394C683BDDEA9A700085AC7
:10DE700026F7FCB3945311270139CEB3964FAB006C
:10DE8000088CB41626F8B1B416270139B6B3944CF1
:10DE9000915026064A9150270139CEB396A600BD6F
:10DEA000F0CE088CB41626F5393CBDDEB93827040F
:10DEB000BDFB313938387EDDF1CE01F4BDFAF727EC
:10DEC000013996431A914327F90926F0393CBDF8E8
:10DED00004961784CF971784BF971786FFB7719B57
:10DEE000D6BBC408FAF8BDBDF8E71A0FCEDF07FFAE
:10DEF00001100E387EEEF730CC0032A702E701CCDD
:10DF0000F004ED057EDFAAB6719B26037EDFA7F63F
:10DF1000718FC4074FC3F8BD1896BB8408AA008A46
:10DF200002BDF8FEFA717FFD7196FC7196DDBCFCB6
:10DF30007191054C810824BF9A1718FC7192847F57
:10DF4000C34000189717DCBCED0071F817FC719204
:10DF5000C30002FD7192F67191C900F77191F171E0
:10DF60008525162608FC7192B37186250CFC718AF2
:10DF7000FD7192B67189B77191DE6C08DF6C7A0021
:10DF8000B82619DC42C30001DD42DC40C90089002B
:10DF9000DD4096AE890097AE96B797B8717F1BFEAD
:10DFA000718227026E003BBDF815CEFB9CFF01106D
:10DFB00020C738CC00017EF0047EF38ABDEEFD243C
:10DFC0000ABDEF65964427F1CC0052FD73AA3C18B8
:10DFD000EC0026DEEC02FD73AC38862CBDEEE026AC
:10DFE000D87EDFF8863BBDEEE027F63CFE73AAFC48
:10DFF00073ACED02387EEEF7CCE225DD46BDEEF0E7
:10E00000DF483CDE46A100260908DF463808A600A6
:10E0100020F0A6002B1908A6002AFB0808A6002657
:10E0200004387EF38ADF4638DE48A6007EE0023CF4
:10E0300016584FC3E20F18EC00186E0038A601BD49
:10E04000E203387EDFE438A601BDE20338BDE40711
:10E05000DC5227037EF004DC542718830001B373DD
:10E06000AC4D2606C18024EC200881FF26E6C18045
:10E0700025E217BDE2037EDFE438A60138E600C1E1
:10E08000412706C14226058B100820E736BDE4076C
:10E09000BDE1CA270C328B30BDE203BDE1E47EDF77
:10E0A000E432BBC431BDE203BDE1EF7EDFE438A65C
:10E0B000013836BDE407DC5227037EF004DC544D02
:10E0C00026F837862CBDEEE027037EF38ABDE407F1
:10E0D000DC5226E6DC544D26E1BDE1CA2616DF46B9
:10E0E000183332BDE20317BDE2031817BDE203DEA9
:10E0F000467EDFE4DF461833328B107EE0E338A63D
:10E1000001387EE08C38A60138E600C1412709C1FC
:10E110004227037EF38A8B4036088623BDEEE02635
:10E120002EBDE40732BDE203BDE1EF7EDFE438A699
:10E13000013836B6C42D802BBDEEE02612BDE407B3
:10E1400032BDE203BDE1E47EDFE438A6013836BD2E
:10E15000E407BDE1CA260C328B20BDE203BDE1EF2E
:10E160007EDFE49654270C328B30BDE203BDE1E440
:10E170007EDFE4328B1020E238A601BDE20338BD19
:10E18000E407BDE1EF7EDFE438388622BDEEE0260D
:10E1900004167EE19D8627A100260D1608A600081C
:10E1A00011270BBDE20320F5BDE407BDE1EF862C8E
:10E1B000BDEEE027D57EDFE43838BDE407BDE1E4FD
:10E1C000862CBDEEE027F37EDFE4A600B1C42B264B
:10E1D000030820F6812C260B08A600088158270387
:10E1E0007EF38A39DC52260E9654BDE203200EDC03
:10E1F000522706CC00277EF004965426F99655BD8A
:10E20000E203393CFE73ACA70008FF73AC3839E079
:10E210003CE046E079E0AEE0FEE105E12EE14AE1D6
:10E2200078E188E1B84E4F5080014C53524480044D
:10E2300041534C448005544150800654504180075E
:10E24000494E5880084445588009434C56800A532B
:10E250004556800B434C43800C534543800D434C43
:10E2600049800E534549800F53424180104342413B
:10E2700080115441428016544241801758474458F7
:10E2800080184441418019534C50801A41424180CA
:10E290001B5453588030494E53803150554C418067
:10E2A0003250554C42803344455380345458538047
:10E2B0003550534841803650534842803750554C72
:10E2C0005880385254538039414258803A52544908
:10E2D000803B50534858803C4D554C803D574149F8
:10E2E000803E535749803F425241812042524E81E5
:10E2F000214248498122424C538123424343812495
:10E300004243538125424E45812642455181274251
:10E3100056438128425653812942504C812A424D0E
:10E3200049812B424745812C424C54812D42475410
:10E33000812E424C45812F4E45478240434F4D82AE
:10E34000434C53528244524F528246415352824769
:10E3500041534C8248524F4C8249444543824A497A
:10E360004E43824C545354824D434C52824F414948
:10E370004D83614F494D836245494D836554494DF5
:10E38000836B4A4D50844E535542448683414444E6
:10E390004486C3435058868C4C444486CC4C4453EA
:10E3A000868E4C445886CE5355428580434D5085C9
:10E3B000815342438582414E448584424954858538
:10E3C0004C44418586454F52858841444385894F59
:10E3D0005241858A414444858B5354414187875338
:10E3E00054414287C7535453878F4A5352878D53A2
:10E3F000544487CD53545887CF425352888D44425A
:10E40000890044578A0000BDE437F6C431A60008ED
:10E410001127FA817C27020939DC543736DC523760
:10E4200036BDE43732339A52DA53DD5232339A54DE
:10E43000DA55DD547EE40ABDE467F6C42BA6000875
:10E440001127FA812627020939DC543736DC523786
:10E4500036BDE46732339452D453DD523233945490
:10E46000D455DD547EE43ABDE50DA60008B1C43AAA
:10E4700027F809813C2504813F250139DC543736D2
:10E48000DC523736CCC651DD527EC885BDE4D2257C
:10E490000B860197552008BDE4D226F57F00557FF5
:10E4A00000547F00537F005239BDE4D227EE25ECA3
:10E4B00020DFBDE4D227DA25D820E1BDE4D226DC76
:10E4C00020CFBDE4D224D520C83233DD523233DD33
:10E4D0005439DF4E381838DF5038183C183CDE50BD
:10E4E0003CDE4EBDE50D3233DD463233DD48964627
:10E4F0009852182A0CDE529C462610DE549C48186E
:10E5000039DE469C522604DE489C541839862DBDBF
:10E51000EEE02606BDF0837EE566862BBDEEE0BD0F
:10E52000E577862BBDEEE02635DC543736DC5237F6
:10E5300036BDE5773233DD463233DD48DC54D3482F
:10E54000DD54DC52974ED9479946DD52964E984697
:10E550002BD0964E98522ACACC00097EF004862D04
:10E56000BDEEE0270139DC543736DC523736BDE5E5
:10E5700077BDF06B7EE534BDE60B862ABDEEE02666
:10E5800021DC523637DC543637BDE60B3332DD48FA
:10E590003332DD46BDF228DC4EDD52DC50DD547EE8
:10E5A000E57AA600812F270581252701393C087FC0
:10E5B00000447D00522A067C0044BDF06BDC5236DC
:10E5C00037DC543637964436BDE60B3297447D002F
:10E5D000522A067A0044BDF06BDC52DD46DC54DD85
:10E5E000483332DD543332DD523CBDF14A381838FD
:10E5F00036A60081252608DE4EDF52DE50DF54327B
:10E600001896442703BDF06B7EE57A0908A60081C1
:10E610002027F981302504813A25308128273E8141
:10E62000262728A6018141250C815B2408CCC5CF73
:10E63000DD527EC885BDEEFDDD52251E3C0FDE524B
:10E64000EC00DD52EC020EDD543839BDEF65964426
:10E650002708398628BDEEE027047EF38A08BDE44A
:10E66000078629BDEEE026F239BDE65396522A030D
:10E67000BDF06B96522B0139CC000A7EF004BDE64A
:10E6800053DC522706CC000B7EF0043C8D0838DDAD
:10E69000545F4FDD5239DE548C000B250A9D9F38A4
:10E6A00038CC000B7EF00418BDF80F3918FE73AAA1
:10E6B0003CDE643CDE663C188628BDEEE02629BDC3
:10E6C000CF737F00527F00537F0054862CBDEEE055
:10E6D00026288623BDEEE0260FA600088134270BEE
:10E6E00081322711813127127EF38ABDF11A9752A8
:10E6F000BDF11A9753BDF11A9754BDF11A97553CC5
:10E70000FE73AADC66ED02DC64ED00381838DF66C3
:10E7100038DF6438FF73AA188629BDEEE026C939B0
:10E720009DA23838CC000C7EF0048628BDEEE02691
:10E7300057BDF083DC54053736BDE407DC52270CA7
:10E74000CC000C7EF0043C8DD7382021DC544D26C3
:10E75000F5C10E24F1C108243386805D2704445A94
:10E7600020F93643948B9720978B329415270732E4
:10E7700033C3000120023233DD54862CBDEEE02786
:10E78000B38629BDEEE027037EF38A39C008868070
:10E790005D2704445A20F9B1C43A24024444364364
:10E7A000948A9701978A32940320C2BDE653965209
:10E7B0002A06CC000D7EF004CC0000DD46DD48DDED
:10E7C0004EDD50DD4CCC4000DD4A860F975ADC48C8
:10E7D000D350DD58DC46D94F994EDD56DC58D34C2A
:10E7E000DD58DC56D94B994ADD5674004E76004F01
:10E7F000760050760051DC529356251E2606DC54D6
:10E8000093582516DC56DD46DC58DD48DC50D34CE9
:10E81000DD50DC4ED94B994ADD4E74004A76004BF0
:10E8200076004C76004D74004A76004B76004C76AC
:10E83000004D7D005A2609DC4EDD52DC50DD543996
:10E840007A005A2089BDE653DC522706CC000E7EA2
:10E85000F0043CDC54040453D74E16584FC3E887E9
:10E8600018EC02DD46EC0093469748964E3D9749DA
:10E870009648D64E3DDB498900D346DD542A067AB8
:10E8800000527A0053383940D840D835482E86296E
:10E89000F4268423C8217A1F7C1DC41C341AD6197F
:10E8A0008C1856173E163A1540145A137412A211BA
:10E8B000D01108104A0F960EE20E2E0D840CDA0CC1
:10E8C0003A0B9A0AFA0A5A09C40924088E07EE0775
:10E8D0005806C2062C058C04F6045603C003200219
:10E8E0008001D6012C0082FFD8FF1AFE5CFD9EFC41
:10E8F000CCFBF0FB0AFA10F90CF7E0F6A0F524F3D4
:10E9000076F15AEE80EA20EA20BDE6533C7D0052C3
:10E910002A09DC545343C38001DD54DC54847FDD79
:10E9200052188C4000182505CC80009352DD461605
:10E930004F05C3E9DE18EC00DD48EC02A300974E5A
:10E9400096473D97517F0050D64E96473DD350D3C2
:10E95000487F00527F00537D00542A1543537300B3
:10E9600052730053C3000118DC52C9008900DD5204
:10E9700018DD543839BDE6533C7F00567D00522ADD
:10E9800006BDF06B7A0056DC52270738CC000F7EAC
:10E99000F004DC5427462BF3CEE9DE7F0057EC0071
:10E9A000189C5418240708087C005720F1DD4A09F8
:10E9B00009EC00DD4CDC4A934CDD48CE0000DF461C
:10E9C000DC54934CDD537F0055BDF14A96574A5FA6
:10E9D000D354DD547D00562703BDF06B3839000059
:10E9E00003240648096A0C8C0FAB12C815E218F90B
:10E9F0001C0B1F1A2223252828262B1F2E1030FB24
:10EA000033DE36BA398C3C563F1741CE447A471C28
:10EA100049B44C3F4EBF5133539A55F558425A8230
:10EA20005CB35ED760EB62F164E866CF68A66A6D9E
:10EA30006C236DC96F5E70E2725473B575047641D4
:10EA4000776B788479897A7C7B5C7C297CE37D890F
:10EA50007E1D7E9C7F097F617FA67FD87FF57FFF2B
:10EA6000CC0002DD545FDD5239CC00DFDD547F0085
:10EA7000527F005339CC000020F2CC00107EF0040D
:10EA8000BDE653DC5226F3965426EFD655BDF083EF
:10EA90005D27E7C12124E386BF948A9701978A9670
:10EAA0008B8A14978B972071EB15721015201278B2
:10EAB000005579005479005379005272041571FBA6
:10EAC000157B400327037C00555A26E339CC0011FF
:10EAD0007EF004BDE653DC5226F3DC5427403C189C
:10EAE000968A84FE9701978A867EB70109CCEB1F30
:10EAF000FD010A7F00547F005596431A914327FB7E
:10EB000001010101D608DC0D9643C6120FD7080E8D
:10EB10001A914327F796430926F27F000838399661
:10EB20000884EF9708DC0DDC54C30001DD54DC528F
:10EB3000C9008900DD523B9608DE4A08DF4A84E2BC
:10EB40009708DE0DDF54B4C42B270EDE548C8000F2
:10EB50002407DE5208DF52DC093B960820F47EF3DE
:10EB60008ACC00127EF0048628BDEEE026F0BDE4DB
:10EB700007DC5226ECDC5427E8183C18862CBDEE46
:10EB8000E026DBBDE407DC5226D7DC5427D3DD4E7C
:10EB9000183818DD508629BDEEE026C23C968A84DE
:10EBA000FE9701978A867EB70109CCEB37FD010AF3
:10EBB000867EB70103CCEB5AFD01047F004A7F003B
:10EBC0004B7F004CC602D708D608DC0DDC09964303
:10EBD000C6160FD7080E1A914327099643DE4E0931
:10EBE0002731DF4E0FDE4A092611964C260D7C0098
:10EBF0004CDE52DF46DE54DF4820D79C5026D30E31
:10EC00007F0008DC549348DD54DC52D2479246DD45
:10EC10005238397F0008CC0000DD52DD543839BD50
:10EC2000E6537F005ADC522A06CC00137EF0043CE7
:10EC300027157400527600537600547600557C00F8
:10EC40005ADC5226ED2011DC5427DE2B0B780055C0
:10EC50007900547A005A20EF7F00467F0047DC5449
:10EC6000C3B172DD487C0047CCB172DD52CC17AD28
:10EC7000DD54BDF14ADC54DD567F0058DC4FDD52D7
:10EC8000965197547F0055BDF14ADC54D357DD5758
:10EC9000965689009756965680809756DC5805DD23
:10ECA00058DC565949DD56730056DC574353C300B0
:10ECB00001DD57965689009756CE0000DC56DD548C
:10ECC000DD482A03CEFFFFDF52DF46BDF228DC4ECF
:10ECD000DD5EDD54CC994BDD48CC0000DD46DD52D5
:10ECE000BDF228DC4EC3F622DD54DC5EDD48CC00EC
:10ECF00000DD52DD46BDF228DC4EC3E2A8DD60CC6B
:10ED00000002DD5EDC57DD544FD6562A0286FFDD59
:10ED100052DC54363705DD58DC5236375949DD565A
:10ED2000CC0000DD46974896609749BDF228DC4F3D
:10ED3000D358DD58DC56C9008900DD564FD64E2A1F
:10ED40000286FFD356DD56D661D7493332DD5233C2
:10ED500032DD54BDF228DC4ED358DD58DC56C900F4
:10ED60008900DD564F5F7D004E2A03CCFFFFD3564E
:10ED7000DD56DC5783875DDD539656820097524FF0
:10ED8000965A9B529752DC53DD5436374FD6522A4F
:10ED90000286FF3637DD5286B19749CC0000DD464A
:10EDA0009748BDF228DC4EDD56DC50DD58C672D7E0
:10EDB000493332DD523332DD54BDF228DC4ED357B5
:10EDC000DD548600D6562A0286FFC90089007D00E0
:10EDD0004E2A03C3FFFFDD523839BDE653DC522B08
:10EDE0000B83000A2506CC00147EF004DC52DD56AD
:10EDF000DC54DD58DC53DD5496529753CC0001DDD2
:10EE000046CC62E4DD48BDF228D64E2A0CC1F0247F
:10EE100008CC0000DD52DD54394F5CD75A2A0286F7
:10EE2000FFDD5416DD52CCB172DD487F00467F0015
:10EE300047BDF228DC509358DD54DC4ED257925631
:10EE4000DD52DC524756DD5EDC544656DD608607F7
:10EE5000975B3CCCFFFFDD52CCFFF3DD54CEEEC41C
:10EE6000BDEE907A005B26F8965A2B13270F780098
:10EE7000557900547900537900524A26F138397790
:10EE800000527600537600547600554C26F13839FE
:10EE9000DC5EDD46DC60DD48BDF228965048DC4E85
:10EEA0005949DD54CC00007D004E2A03CCFFFFDD24
:10EEB00052EC02D354DD54EC00D9539952DD520880
:10EEC000080808390000005BFFFFFDDE00000AAB08
:10EED000FFFFD55500008000FFFF0000000100008B
:10EEE000160908A600812027F90811270109390809
:10EEF000A600812027F939BDF3657EF38A0908A6AB
:10EF000000812027F9813F262608A600812027F9C5
:10EF100081282705CC00400C39BDE653DC5226275A
:10EF2000DC544D2622C106241E0505C373B039806A
:10EF300040240139262008BDE653DC522609DC5462
:10EF400018BC7288182506CC00027EF00405054323
:10EF500053C372190C39811B25020D390848481614
:10EF60004FC3721839BDF0837F0044BDEEF07F00BF
:10EF700046812626037EF0258130240139813A25F9
:10EF80000139840F7D0044260A7C0044975508A669
:10EF90000020E57C0044D644C10524149747DC5486
:10EFA00005DD540505D354D346DD5408A60020C81A
:10EFB0009747DC5405DD54DD50DC5259492B42DDC6
:10EFC00052DD4E78005179005079004F79004E2B78
:10EFD0003078005179005079004F79004E2B22DCB7
:10EFE00054D350DD54DC52D94F994E2B14DD52DCF2
:10EFF00054D346DD54DC52C90089002B04DD522075
:10F00000AACC00033CCEF00B7EF390484F573F2034
:10F01000204552524F52202300574841543F0D5330
:10F020004F5252590D08A6008148270909399644C4
:10F03000260209093908A600803025F2810A250A2E
:10F040008007810A25E8811024E47C0044D644C16D
:10F050000924AEC60478005579005479005379002C
:10F06000525A26F19B5597557EF035730052730026
:10F0700053DC544353C30001DD54DC52C900890002
:10F08000DD52397F00527F00537F00547F00553995
:10F090003CFE738C3CCEF0B8FF738CBDF0CE38FFD5
:10F0A000738C38393CFE738C3CCEF0B8FF738CBD4A
:10F0B000F11A38FF738C383900010044415441463D
:10F0C000494C45204F56455252414E4745003CBDA4
:10F0D000F0D43839367D00642609DC6505250481C5
:10F0E000072506CC00047EF004331807360F18D726
:10F0F000BC4C9A179717DC66847FC340001896BCF7
:10F10000A70071F81716320637DC66C30001DD660A
:10F11000DC64C9008900DD6432393CBDF120383936
:10F120007D00642609DC6505250481072506CC00E1
:10F13000057EF0041607365C170F9A179717DC66E2
:10F14000847FC3400018A60020B8DE46264BDE4868
:10F1500026083838CC00067EF004DE52263BDC540C
:10F16000CE00007C005278004979004824F57600F2
:10F170004876004993482404D3482001087A005275
:10F18000270B18051874004876004920E7DF54CE95
:10F190000000DF52DF4EDD50397F004ADE52DF4E85
:10F1A000DE54DF50CE0000DF52DF547C004A78008E
:10F1B0004979004879004779004624EF7600467681
:10F1C0000047760048760049DC509348DD50DC4E1D
:10F1D000D2479246DD4E2410DC50D348DD50DC4E41
:10F1E000D9479946DD4E20127C0055240D7C0054F1
:10F1F00024087C005324037C00527A004A271A78A2
:10F200000055790054790053790052740046760015
:10F210004776004876004920AF393CCE004686103C
:10F220006F00084A24FA38397F00447D00522A06CC
:10F230007C0044BDF06B7D00462A1A7A00447300BE
:10F2400046730047DC484353C30001DD48DC46C930
:10F25000008900DD46BDF27E964E2A06CC00077E70
:10F26000F0049644271773004E73004FDC5043534D
:10F27000C30001DD50DC4EC9008900DD4E397F003E
:10F280004E7F004F9649D6553DDD50D655272F96D7
:10F2900048270B3DD34FDD4F964E8900974ED655EC
:10F2A0009647270A3DD34EDD4E24037EF33CD655C8
:10F2B0009646270A3D4D26F3DB4E25EFD74ED65412
:10F2C00027389649270B3DD34FDD4F964E8900973F
:10F2D0004ED654964827083D4DD34E25CEDD4EF6EA
:10F2E000C42FC1452614D6549647270A3D4D26BB48
:10F2F000DB4E25B7D74E964626B1D65327239649DF
:10F3000027093DD34EDD4E2533974ED653964827D9
:10F310000A3D4D2627DB4E2523D74E96479A462693
:10F320001BD65227169649270A3D4D260FDB4E2540
:10F330000BD74E96489A479A46260139CC00077E4D
:10F34000F004BDEEFD25433736863DBDEEE0263A9E
:10F35000BDE407DF46380FDC52ED00DC54ED020E51
:10F36000DF52DE4639863ABDEEE0260532327ECBEC
:10F3700014860DBDEEE026063232087ECADE39BDA7
:10F38000EEF0810D27F8813A27F43C4F5FCEF0195B
:10F390000EDD547F00527F0053CCFB6EDDAC7F004E
:10F3A000B57D008127273CFE738C8CFFFF38271D1D
:10F3B00096B681182606BDFB6E7F00B68EBFFFCCC9
:10F3C0000000FD738EFD7394DE82BDCAEC7F00B336
:10F3D0007F00B496B6270CBDFB6E96B68118260347
:10F3E0007F00B64FBDF528860AB7B59ADC542709C9
:10F3F0007F0045BDF563BDF6A7FE738C8CFFFF262D
:10F40000037ECDF4EC0026037EC706BDF5FD18385B
:10F4100009DF4618A600810D270FBDF6A99C4626D8
:10F4200005863FBDF6A90820EBBDF6A97EC7063CC0
:10F43000CEF01F4F5F7EF390C60DD74636DF5218D1
:10F44000C300F0DD54DE52BDFB31817F27418108CE
:10F45000273D810A27F1810027ED810326113337EB
:10F46000C13A260B33383838FF738C387EF6CAA77A
:10F4700000089146261233C13A270CBDFB6E810D60
:10F480002605860ABDFB6E39BDFB6E9C5426B89CD2
:10F490005227B4098608BDFB6E8620BDFB6E860828
:10F4A000BDFB6E20A2DE548C80002508CC00087EB7
:10F4B000F0043232CE73D2BC73A225040D86FF391C
:10F4C000EC00847F9354250139E602DF564FD35672
:10F4D0001820E4200108A6002AFB20DB3CDE52278E
:10F4E0000738CC00087EF004DE548C800024F2FE45
:10F4F000738CEC00847F26035D27B7189C54382555
:10F50000D2FE738C200C09E6000886FF50DF56D32C
:10F510005618DC548A80A1002605E1012601398CA9
:10F5200073D226E20D86FF3916A60008112601398E
:10F530003637BDF6A93332810D26EE398622BDEE6F
:10F54000E0260ABDF528810D2601094F398627BD21
:10F55000EEE027EF817F260A81082606860D9DAB07
:10F5600020E9393C964536848097449645847F97B8
:10F57000458614367A0045F6B59AC10A260E7D00F6
:10F58000522A09BDF06B7C00447A0045F6B59A4FCB
:10F5900018DF487F00477F0046BDF14ADE5226044F
:10F5A000DE542708D651377A004520E0D651377B04
:10F5B00080442715964484012704862D9DAB7A004C
:10F5C000452B1B86309DAB20F57A00452B06862007
:10F5D0009DAB20F5964484012704862D9DAB328196
:10F5E00014270C810A25028B078B309DAB20EF324C
:10F5F00097453839BDF5FD4FBDF5280839EC008435
:10F600007FDD547F00527F00530808088604974529
:10F61000BDF5638620BDF6A939FE73A4BC73A82688
:10F620000139A600083CFE73A6A70008FF73A638A0
:10F6300020EAFE73AABC73AE26013909A6003CFE7F
:10F6400073AC09A700FF73AC3820EA3233DF5E38B1
:10F65000FF7394271838FF739A38FF739C38FF7331
:10F660009638FF739838FF739E38FF73A03736DEE5
:10F670005E393233DF5E308CB6012405DE5E7EF407
:10F680002FFE7394271BFE73A03CFE739E3CFE73FB
:10F69000983CFE73963CFE739C3CFE739A3CFE7352
:10F6A000943C3736DE5E39860D369DAB3236810DA1
:10F6B0002604860A9DAB32397D00932601397D00F0
:10F6C0009E27FA7F0093BDFACF0E7D008C271A8EFD
:10F6D000BFFDCC0000FD738EFD7394CC0064DD543F
:10F6E000CC0000DD523C7ECB23FE738C2727CEF767
:10F6F00018BDF6A74FBDF528FE738CEC00847FDDA6
:10F70000547F00527F00537F0045860AB7B59ABDEB
:10F71000F563BDF6A77EC706425245414B204154D2
:10F72000204C494E4520000F36BDF80432843F8AF4
:10F730008016BDF75371DF17BDF7CED756BDF7CE94
:10F74000D757BDF8150E200439BDF75371DF177177
:10F75000BF173971DF1771BF1771EF17724017723A
:10F76000201771DF177210177220178608BDF7F186
:10F77000390F3632843F36C630BDF74932368AC03B
:10F7800016BDF753BDF7A80E01010F32843F8A4022
:10F7900016BDF753D656BDF7EFD657BDF7EFBDF7F9
:10F7A000A8C600BDF7490E3971EF1771DF1771BF99
:10F7B00017CE04C47220170101010171DF17092659
:10F7C000F372401772201771DF1771BF1739C60225
:10F7D00072201771DF177B081727015C72201758FA
:10F7E00024F171DF177B081727015C722017398617
:10F7F000085871DF17721017250371EF1772201761
:10F800004A26EE399617844797178A40971739BDCD
:10F81000F804BDF8447B02BB271E7B04BB271E3CBB
:10F8200018C601BDF8E772201771DF177220177133
:10F83000DF177240171838397B04BB26067187170B
:10F84000728017390F3C1896171684CF971784BF0C
:10F8500097177B02BB27037EF8C51853CB08860495
:10F86000C1082505721017200371EF177220177158
:10F87000DF1758C40F4A26E8961716CA20D71797DD
:10F8800017D7179717D7179717D7179717D7179708
:10F8900017D717BDF921CE00040901010101012686
:10F8A000F8CE000A4F5F057B08172702CB40722075
:10F8B0001771DF170926EF724017380E39F4B4E4D8
:10F8C000A4D494C484184FC3F8BD18D6BBC408EAA6
:10F8D00000BDF8E786104A26FD8602BDF8FE368692
:10F8E000104A26FD3220D3860858240572101720AE
:10F8F0000371EF1772201771DF174A26EC39CE001B
:10F900000C5F052405721017200371EF177B081791
:10F9100027015C72201771DF170926E6050505052A
:10F9200039CE00050926FD971739961784CF97170A
:10F9300084BF9717D6BBC408FAF8BDBDF8E7368672
:10F94000104A26FD320F3C7C0053D6534FC3F8BDFE
:10F950001896BB8408AA008A02BDF8FE0E38BDF9CD
:10F96000F1D653D15226DE7EF81A9752D7467F0041
:10F9700053BDF8047B02BB27037EF92A0F3C71EFCD
:10F980001771BF1772201771DF17721017CE000999
:10F9900072201771DF170926F7CE00030901010154
:10F9A000010126F87C00539653438B089754CE00F0
:10F9B0000A4F5F71DF177800547B105427057210CF
:10F9C00017200371EF17057B081727015C722017BA
:10F9D0000926E071DF170E38050505050505BDF997
:10F9E000F19652915327043C7EF9997240177EF8A4
:10F9F000387D004627167A004626057C00462008FA
:10FA00007C004637BDF0CE32BDF0CE3905057B0215
:10FA1000BB27F5050520F1961E84D0275584502775
:10FA20000396123BDE719612A7007B0176271281A6
:10FA3000132605728076203A81112605717F762083
:10FA400031810326037C0093098C728B2603CE73CD
:10FA50008BDF717D0075261A189373C1402613FC45
:10FA6000B596B3B594C1FF27098613BDFB6E86FF1B
:10FA7000977596118424812427013B7B01762723E7
:10FA80007B8076271EDEAFBDF6B871FB110E01013B
:10FA900096431A914327F90F0927057B807626E7BD
:10FAA000717F76FEB596A600098CB4932603CEB579
:10FAB00093FFB5967D007726029713FEB596BCB5E9
:10FAC00094260471FB113B7204113B86FF97753C31
:10FAD000CE738BDF71DF7371FB11CEB593FFB594DD
:10FAE000FFB596967527088611BDFB6E7F007538A9
:10FAF000717F767F0093399674907239B6B597B05E
:10FB0000B59539DE643CDE663CDEB3EC00DD64ECCA
:10FB100002DD663CBDF11A38D664E700D665E70120
:10FB2000D666E702D667E70338DF6638DF64333826
:10FB3000393C3736DCB33226CADE739C7126031A91
:10FB400020F7A60036098C728B2603CE738BDF73E9
:10FB50009675270F189371C14026088611BDFB6E5C
:10FB60007F0075323338810326037A0093393C379E
:10FB700036FCB596B3B594C1FF27F6FEB59432A70F
:10FB800000098CB4932603CEB593FFB5947204118B
:10FB900033383986209DAB86209DAB39DE6C08DF7B
:10FBA0006C7A00B82619DC42C30001DD42DC40C992
:10FBB000008900DD4096AE890097AE96B797B87180
:10FBC0007F1B3B3B3B8E00FD86029790BDFBDF1AFF
:10FBD0001A1ACE0000DF42DF407F00AE7EC68B8661
:10FBE00012971B7F00017F008A7F00207F008B8699
:10FBF0000A97118605971086E09714864097178616
:10FC0000F797169770860B97BBBDF80F86029790F3
:10FC1000860397707F009186FF9780867EB7010FDD
:10FC2000CCFB9CFD0110865F7B01BB270286BF9742
:10FC30001C9763860197B897B772401B0E86FF9793
:10FC400077392A202050433D2420413D2420423D45
:10FC50002420463D2420583D242040583D24205354
:10FC6000503D24204024DEAC3CCEFB6EDFAC0E8643
:10FC70000DBDFB6E860ABDFB6ECEFC42BDFCFE3C9C
:10FC800030EC091809BDFD0638BDFCFE3C30A60667
:10FC9000BDFD0B38BDFCFE3C30A605BDFD0B38BDDF
:10FCA000FCFE3C30A604BDFD0B38BDFCFE3C30EC38
:10FCB0000718BDFD0638BDFCFE3C30EC0718EC0013
:10FCC00018BDFD0638BDFCFE3C3018C3000A18BD47
:10FCD000FD0638BDFCFEFE7282BDFD06863DBDFB05
:10FCE0006EFE7282860836A60008BDFD0B8620BD1A
:10FCF000FB6E324A26F038DFAC3BBDFB6E08A60037
:10FD0000812426F608393C328D013236444444447D
:10FD10008D0132840F8B30813A25028B077EFB6E7A
:10FFC7007EFAFC7EF8447EF8047EF8157EF0907E7B
:10FFD700F0A47EFAF77EFB317EFB6E7EFACF7EF8C9
:10FFE7000F00DF0100010FFBC3FA17010301060130
:09FFF70009010CFC66FBC4FBC50A
:00000001FF
